:1000000051C0000001C058C0032F36B3032701FDC3
:1000100005C002FD8BC032FF92D0189512B602BE09
:10002000423081F103E003BF32FF40E0413019F07C
:1000300032FD7EC084D0213029F090F431FD3CC0E7
:1000400021E0189531FFC1F5012D0531A8F50430E7
:1000500098F1212C312C269425E055241DE018958B
:10006000121850F11318D0F1131430F5263020F186
:1000700001E020FB551C441C50F820271A9549F03C
:10008000A2F51AC031FFC09831FDC09A32FF11C0ED
:100090001895253011F0273041F5461027C057102C
:1000A00025C00DC000E808B900E605BF00E20BBF9F
:1000B000002440E06624772436B301E007BB08BA89
:1000C00032FF40E0413011F032FD32C020E003BE8B
:1000D00002E008BF09BF78948895FECF03E0253081
:1000E00021FFC7CF20271123A1F21895642C752C6E
:1000F000042D077F0731C1F4052D0D3BA9F44130D4
:10010000A9F005E003BF02BEC39ABB9A02B7003B49
:10011000B29BE0F341E0BB980EE202BE12B613942C
:10012000E9F70A95D1F7C8CF403049F232FFC1CF85
:1001300001E007BB08BB42E066247724C7CF34FF49
:0E01400003C0C39ABB9A0895BB98C398089554
:00000001FF
